:020000040000FA
:020000003128A5
:080008000B1D09000B11200083
:1000100045089500C30A4302031C0900C3010130CF
:10002000C406441C2328250006309600200033080F
:1000300025009100250002309D0020003408250095
:1000400098002000090025000630960025000030A9
:100050009100250002309D0025000030980020000E
:10006000090021007A30990023008C0123008D01C2
:10007000210004308C00210000308D0020008C0114
:1000800020008D01210006309500200045089500D4
:100090000B110030C3008B1625000C309300250097
:1000A0000C309A00250004309E0022001D109D1483
:1000B0001D159D151D16200004309C0028000430DD
:1000C000970000308E23B60001308E23B30002303B
:1000D0008E23B40003308E23B50009308E23C50073
:1000E0000C308E23A9000D308E23AA000E308E23F3
:1000F000AB000F308E23AC0010308E23AD001130DA
:100100008E23AE0012308E23AF0013308E23B0004A
:1001100014308E23B10015308E23B20020008C01E4
:100120008D01BA0108308E23B700512AA201A30124
:10013000A401A501A601A701A001A1010C19B128E4
:100140000C19B3280030200203199E282030200209
:100150000318B728A10A0C3021020319BA28A001FC
:100160009E280000000000000000A00A9E28A001B8
:10017000A1019E28A001A1010C19CA280C19CC28A4
:10018000003020020319BC28203020020318D02898
:10019000A001BC280000000000000000A00ABC284C
:1001A00096019701A001A101A1150C19E8280C19CD
:1001B000EA28003020020319D52820302002031835
:1001C000EE28A20D2214A10BE628F228A001D528C2
:1001D0000000000000000000A00AD528A20D221097
:1001E000A10BE628A001A1010C1902290C19042970
:1001F000003020020319F4282030200203180829B7
:10020000A00196280000000000000000A00AF428C9
:10021000A001A101A1150C191E290C1920290030DB
:10022000200203190B292030200203182429A30DD2
:100230002314A10B1C292829A0010B290000000070
:1002400000000000A00A0B29A30D2310A10B1C29FC
:10025000A001A1010C1938290C193A2900302002FB
:1002600003192A292030200203183E29A0019628CC
:100270000000000000000000A00A2A29A001A1013E
:10028000A1150C1954290C19562900302002031904
:1002900041292030200203185A29A40D2414A10B4F
:1002A00052295E29A0014129000000000000000041
:1002B000A00A4129A40D2410A10B5229A001A101DB
:1002C0000C196E290C1970290030200203196029BD
:1002D0002030200203187429A001002A0000000029
:1002E00000000000A00A6029A001A101A1150C19BD
:1002F0008A290C198C290030200203197729203013
:10030000200203189029A50D2514A10B88299429F2
:10031000A00177290000000000000000A00A772952
:10032000A50D2510A10B8829A001A1010C19A42954
:100330000C19A6290030200203199629203020022A
:100340000318AA29A001002A0000000000000000F4
:10035000A00A9629A001A101A1150C19C0290C1908
:10036000C229003020020319AD29203020020318D1
:10037000C629A60D2614A10BBE29CA29A001AD29A4
:100380000000000000000000A00AAD29A60D261004
:10039000A10BBE29A001A1010C19DA290C19DC2935
:1003A000003020020319CC29203020020318E02954
:1003B000A001002A0000000000000000A00ACC29D3
:1003C000A001A101A1150C19F6290C19F82900307A
:1003D00020020319E329203020020318FC29A70D6D
:1003E0002714A10BF429002AA001E3290000000032
:1003F00000000000A00AE329A70D2710A10BF42993
:10040000220823062406250626062706031D96280D
:100410002308FE39A80022082906031D192A2808E6
:100420002A06031D192A2318172A3710512A3714B0
:10043000512A22082B06031D272A28082C06031DF3
:10044000272A2318252AB710512AB714512A22081F
:100450002D06031D352A28082E06031D352A2318CC
:10046000332A3711512A3715512A22082F06031D26
:10047000432A28083006031D432A2318412AB711AE
:10048000512AB715512A22083106031DCD2A280802
:100490003206031DCD2A23184F2A3712512A371648
:1004A000512A1F3036060319692A293036060319E6
:1004B000732A2A3036060319812A2B30360603198F
:1004C0008F2A333036060319A12A34303606031931
:1004D000B32A37186D2A0F24C92AB718712A39246C
:1004E000C92A7B24C92A3718772A0F24C92AB718A2
:1004F0007B2A2424C92A37197F2A3924C92A7B2434
:10050000C92A3718852A0F24C92AB718892A3924F5
:10051000C92A37198D2A4E24C92A7B24C92A37189B
:10052000932A0F24C92AB718972A3924C92A3719B8
:100530009B2A4E24C92AB7199F2A6424C92A7B24DE
:10054000C92A3718A52A0F24C92AB718A92A24248A
:10055000C92A3719AD2A3924C92AB719B12A4E2414
:10056000C92A7B24C92A3718B72A0F24C92AB718E1
:10057000BB2A2424C92A3719BF2A3924C92AB71902
:10058000C32A4E24C92A371AC72A6424C92A7B24BD
:10059000C92A00308E23B60096282209031DD22ACC
:1005A000BA01962822080319772BA21BDD2A70397D
:1005B000703A0319EC2ABA019628BA019628EC3051
:1005C0002302031D9628073024060319992B2508BA
:1005D000BC0024087E238E283A1CDB2AA5080319B8
:1005E000342B2208783A0319FE2A2208743A031998
:1005F0001C2B22087C3A0319242B9628241A9628AF
:1006000023088E23BB000F23BB05A41D0B2B3B0827
:10061000031DF82396283B080319F8239628033076
:100620008A0024080739820701340234043408346C
:10063000103420344034803423088E232402031DD8
:100640009628BA01F823962807302306031D2D2B80
:1006500008302406031DF52B9D2B2408BC0023081D
:100660007E23BA01F8239628221D452BA21896282E
:10067000221C622B3B2B2308B800B8030310B80DD3
:100680000310B80DBA14F8239628BA1C962822082D
:1006900003393807B900073039060319942BA21D16
:1006A000592B2308BC0039087E23B901BA01F8236D
:1006B000962839088E232302031D9628B901BA0112
:1006C000F8239628BA1C9628A21D6E2B2308BC007E
:1006D0001C307E23B801BA01F82396281C308E23E3
:1006E0002302031D9628B801BA01F8239628220890
:1006F0002306031D96283A148D01962823009100A5
:1007000020003C0823009300151555309600AA30B0
:100710009600951495188A2B20000800230091005C
:10072000151413082000080008302306031DF52BBC
:100730009D2B08302506031D96281F30BC00003075
:100740007E23FF30BC0001307E23FF30BC0002302E
:100750007E23FF30BC0003307E230030BC00043019
:100760007E230030BC0005307E235B30BC000630A9
:100770007E239C30BC0007307E230030BC00083054
:100780007E233830BC0009307E238130BC000A3023
:100790007E23F830BC000B307E238130BC000C304F
:1007A0007E23FA30BC000D307E238130BC000E3039
:1007B0007E23FC30BC000F307E238130BC00103023
:1007C0007E23FE30BC0011307E238230BC0012300C
:1007D0007E23F830BC0013307E238230BC001430FE
:1007E0007E23FA30BC0015307E23B8013A108E28E3
:1007F0008D150724072407240724072407248D11B7
:10080000080000000230C000C00B042C0800473074
:10081000C10001240B2CC10B092C000008008B1314
:1008200022008D172500073096002000350825008E
:100830009100250000309D00250000309800280020
:10084000950120009A0108008B1322008D132500CA
:100850000930960020003408250091002500003062
:100860009D002500003098002800950120009A0185
:1008700008008B1322008D1325000B3096002000FA
:10088000340825009100250000309D00250000302F
:1008900098002800950120009A0108008B1322007F
:1008A0008D132500063096002000330825009100A6
:1008B000250002309D002000340825009800280003
:1008C000950120009A0108008B1722008D13250046
:1008D00006309600200033082500910025000230E4
:1008E0009D00200034082500980028009501200074
:1008F0009A01441408008B1322008D132500063042
:1009000096002000330825009100250000309D004E
:100910002500003098002800950120009A01080069
:100920001430BF003230BD00C830BE0000000000EF
:0E093000BE0B962CBD0B942CBF0B922C080016
:020000040001F9
:02000E00A40943
:02001000FF1CD3
:10E000001F00FF00FF00FF00000000005B009C00FD
:10E01000000038008100F8008100FA008100FC0057
:0CE020008100FE008200F8008200FA007F
:00000001FF
